:020000040000FA
:060000000C3003303A2829
:08000800A000030EA100831209
:100010008B1C32288B1032181428B21C3228643002
:10002000010203183128182800001628172818285C
:1000300019281A281B281C281D281E281F283210A2
:10004000B214A810031005190314AA0DA90DA80DC8
:10005000B10B322832152A08AF002908AE00280853
:10006000AD00B21081010B11210E8300A00E200EF5
:02007000090085
:0C007400203084008001840A6030040207
:10008000031C3C281230B10099218316FF239000F5
:10009000831283160C308505870183128501870141
:1000A000073099000030831691009F008312C830FA
:1000B00083168100831231309000003083168C004B
:1000C000831210308B00BD1B6B2885196B286400D0
:1000D000851D6728EF21EA2181018E018F010B1117
:1000E0008B100B108C018B17BC21842032199A20A5
:1000F000B40B8228031085190314BA0DF0303A02AC
:1001000003190D21182275286400321808000B1DF0
:1001100008000B11B21032141230B100051D9528E1
:10012000331483160113831208003310831601174A
:100130008312080032110130B7008B1320303707CB
:1001400083169B001C141A088312A400A500C0305B
:10015000A5061030370783169B001C141A0883125B
:10016000A3000030370783169B001C141A08831263
:10017000A2008B17331CC22822090339A200A3094D
:10018000A409A50922082D02031D072923082E0210
:10019000031D072924082F02031DE128013037021F
:1001A000031DD828D7283E18D8283E143F14BC2158
:1001B00002303702031DE128BE18E128BE143F14A7
:1001C000C42125082F02031DF92801303702031D21
:1001D000EF28EE283E1CEF283E103F14C9210230C4
:1001E0003702031DF828BE1CF828BE103F14D12189
:1001F00007295F08F039A03C0319072933180329A0
:100200002F18072906292F1C07290629D621B70AE6
:1002100003303702031808009D280130B600B400EF
:10022000B500B70085018701B213E3217021842056
:10023000B40B3E29031085190314BA0DF0303A02AD
:10024000031965290C1C35290C10C00A420840020C
:1002500003193329420A4002031970210230370280
:1002600003197021352985018701B50B3E29FA3024
:10027000B5000230370296300319B500321D172938
:100280003211331C48292D090339AD00AE09AF09DD
:100290002F1CB2132F1C1729B21B17292E18172930
:1002A000B2178B1320303707BC002F08BB00862104
:1002B00010303707BC002E08BB00862100303707FE
:1002C000BC002D08BB0086218B1785018701E62124
:1002D000B70AB60103303702031C1729EA210800C8
:1002E0008E018F01C0010C10013037020319D92192
:1002F000023037020319DE2108003F1C08003F10BE
:100300001030BC003E08BB00862108008B133B0860
:1003100083161C159A003C089B0055309D00AA309E
:100320009D009C1464009C1892291C1183128B1749
:100330000800831600309B001C141A088312BD00AD
:10034000831610309B001C141A088312BE008316FB
:1003500020309B001C141A088312C2000130C21BFB
:10036000C200C2080319C200831630309B001C145F
:100370001A088312DF00080005120514400842071E
:10038000D0004108D10008000130CC000130C80085
:1003900008000510051640084207D0004108D100AA
:1003A00008000230CC000130C8000800051005121A
:1003B0000800380911398500B800080038092239C9
:1003C0008500B8000800B80138140800B801B81456
:1003D000B8160800BE18C421BE1CD1210800B60101
:1003E000B401B5013D1CF729BD01BD14F929BD01BA
:1003F0003D143D08B6006400FD29FE29FF29002AAE
:10040000012AB51B8514B51F8510B51B8516B51FB0
:100410008512B40BFB29B50BFB290310B60CB608EB
:10042000031DFB290030BC003D08BB0086210800ED
:100430008F08031908008F013C308E004D094C05D0
:10044000CA004C094D05CB00C80803192D2AFF30FE
:100450003D1CC800C80F402A6322C10A0319C00A04
:100460005F080F390A3C0319080050084002031DB9
:10047000080051084102031C08000510051208007D
:100480004808C9004A188514CA18851649080E027A
:100490000318522A4B188510CB188512FF304802DA
:1004A000031908008F08031D0800842049080E0264
:1004B000031C522A4A188510CA1885124B18851435
:1004C000CB18851608004A188514CA188516CA0163
:1004D0004B188510CB188512CB014C08CD007D211F
:0204E000080012
:0404E20000340034AE
:084000000A000300060009009C
:02400E00CC01E3
:10420000010003000300030003000200020002009B
:1042100002000000000000000000FF00FF00FF009F
:10422000000000000000000000000000000000008E
:104230000000C000C000C000C000FF00FF00FF0081
:104240000100C300F300CF00FF00C300F300CF0064
:10425000FF00C300F300CF00FF00FF00FF00FF00DE
:10426000FF00FF00FF00FF00FF00FF00FF00FF0056
:10427000FF00FF00FF00FF00FF00FF00FF00FF0046
:10428000FF00FF00FF00FF00FF00FF00FF00FF0036
:10429000FF00FF00FF00FF00FF00FF00FF00FF0026
:1042A000FF00FF00FF00FF00FF00FF00FF00FF0016
:1042B000FF00FF00FF00FF00FF00FF00FF00FF0006
:1042C000FF00FF00FF00FF00FF00FF00FF00FF00F6
:1042D000FF00FF00FF00FF00FF00FF00FF00FF00E6
:1042E000FF00FF00FF00FF00FF00FF00FF00FF00D6
:1042F000FF00FF00FF00FF00FF00FF00FF00AA001B
:00000001FF
